:020000040800F2
:1000000000C00020F9020008E51A0008E91A0008FB
:10001000ED1A0008F11A0008F51A000800000000A7
:10002000000000000000000000000000F91A0008B5
:10003000FD1A000800000000011B0008051B000855
:10004000AD170008AD170008AD170008AD17000880
:10005000AD170008AD170008AD170008AD17000870
:10006000AD170008AD170008AD170008AD17000860
:10007000AD170008AD170008AD170008AD17000850
:10008000AD170008AD170008AD170008AD17000840
:10009000AD170008AD170008AD170008AD17000830
:1000A000AD170008AD170008AD170008AD17000820
:1000B000AD170008AD170008AD170008AD17000810
:1000C000AD170008AD170008AD170008AD17000800
:1000D000AD170008AD170008AD170008AD170008F0
:1000E000AD170008AD170008AD170008AD170008E0
:1000F000AD170008AD170008AD170008AD170008D0
:10010000AD170008AD170008AD170008AD170008BF
:10011000AD170008AD170008AD170008AD170008AF
:10012000AD170008AD170008AD170008AD1700089F
:1001300000000000000000000000000000000000BF
:1001400000000000000000000000000000000000AF
:10015000000000000000000000000000000000009F
:10016000000000000000000000000000000000008F
:10017000000000000000000000000000000000007F
:10018000000000000000000000000000000000006F
:10019000000000000000000000000000000000005F
:1001A000000000000000000000000000000000004F
:1001B000000000000000000000000000000000003F
:1001C000000000000000000000000000000000002F
:1001D000000000000000000000000000000000001F
:1001E0005FF8E0F100B583B001F0D0FA304B314A4E
:1001F0001360314A1360314B314A03E011681960D2
:10020000043304322F498B42F8D32A4B1A682E4B01
:100210009A4204D1284B1A682C4B9A4200D0FEE730
:10022000234B2B4A13602B4A13602B4B02E0002216
:100230001A600433294A9342F9D3254B1B6813B93A
:10024000244B1B6803B1FEE701F0ACFA694601A834
:1002500001F094FA224C234B1C1BA410002504E04F
:100260001F4B53F8253098470135AC42F8DC1E4C43
:100270001E4B1C1BA410002504E01B4B53F825301B
:1002800098470135AC42F8DC0099019801F0A4FBD5
:100290000546174C174B1C1BA41004E0013C144BE3
:1002A00053F824309847002CF8DC284601F064FA13
:1002B000BABADECA000000201000002000000020B2
:1002C000B82400081400002078563412325476986E
:1002D00014000020BC01002014000020C0010020F8
:1002E0009403000894030008940300089403000892
:1002F000940300089403000808B5FFF773FF00BFDC
:1003000000BEFEE71EF0040F0CBFEFF30880EFF312
:1003100009807146124A104700BEFEE700BEFEE7A4
:100320001EF0040F0CBFEFF30880EFF30980714655
:100330000C4A104700BEFEE71EF0040F0CBFEFF39F
:100340000880EFF309807146074A104700BEFEE7B8
:1003500000BEFEE700BEFEE700BEFEE770470000FD
:0C03600019030008350300084D030008D5
:10036C00B82400080000002014000020B824000865
:10037C00000000000000000014000020C00100205C
:08038C00000000000000000069
:1003940010B5044600F0C4FF064BA3FB00308009EF
:1003A40000F098F8002221464FF0FF3000F050F89A
:1003B400002010BDD34D621008B5074A136843F0FE
:1003C40010031360032000F025F80020FFF7E0FF7E
:1003D40001F012FB002008BD00200240024A13680D
:1003E40001331360704700BF18000020014B1868E8
:1003F400704700BF1800002010B582B00190FFF7CD
:10040400F5FF0446FFF7F2FF001B019B9842F9D366
:1004140002B010BD10B50446C31E042B03D9BA2183
:10042400094801F0E7FA094AD36823F4E0631B049E
:100434001B0C240204F4E064234343F0BF6343F43D
:100444000033D36010BD00BFB41D000800ED00E010
:1004540070B504460E4615460F2A03D9D2211A4810
:1004640001F0C8FA0F2E03D9D321174801F0C2FABC
:10047400164BDA68C2F30222C2F10701042928BF2D
:100484000421131D062B01D9033A00E000220123A5
:1004940003FA01F101393140914003FA02F2013AC1
:1004A4002A400A43002C06DA04F00F041201D2B2E7
:1004B400074B1A5570BD1201D2B204F1604404F521
:1004C400614484F8002370BDB41D000800ED00E011
:1004D40014ED00E00138B0F1807F0AD2064B586079
:1004E400F021064A82F823100020986007221A603F
:1004F40070470120704700BF10E000E000ED00E00D
:1005040010B50446042805D020B14FF4DF71084823
:1005140001F070FA042C05D1064A136843F0040371
:10052400136010BD034A136823F00403136010BD65
:10053400B41D000810E000E008B501F005FB08BD9B
:100544002DE9F04383B080460F46B54B98421BD04B
:1005540003F58063984217D003F58063984213D063
:1005640003F5806398420FD003F5806398420BD063
:1005740003F58063984207D003F58063984203D063
:10058400CF21A84801F036FA3B881BB9D021A548F1
:1005940001F030FA7B68012B22D9112B20D0022BD9
:1005A4001ED0122B1CD0A04A934219D002F58012FF
:1005B400934215D002F58012934211D0A2F5F8129D
:1005C40093420DD002F58012934209D002F58012B5
:1005D400934205D0032B03D0D121924801F00AFAAB
:1005E4004FF000094E463FE10125B5403C682C40E0
:1005F400A54240F038818A4B98451BD003F58063AF
:10060400984517D003F58063984513D003F58063AC
:1006140098450FD003F5806398450BD003F58063AC
:10062400984507D003F58063984503D0DF217D48C2
:1006340001F0E0F97B68122B49D00CD8022B3AD098
:1006440004D8002B4FD0012B1ED067E0032B60D0C1
:10065400112B24D062E0754A934244D008D8A2F505
:10066400801293423FD002F58032934256D13AE051
:100674006F4A934237D002F58032934233D0A2F5C9
:10068400801293424AD12EE0FB68013B022B03D92E
:10069400E721644801F0AEF9D7F80C903EE0FB681E
:1006A400013B022B03D9EE215E4801F0A3F9FB685C
:1006B40003F1040932E0FB68013B022B03D9F52165
:1006C400584801F097F9FB6803F1080926E0FB6834
:1006D400013B022B03D9FC21524801F08BF9FB6842
:1006E40003F10C091AE0BB68022B04D940F209118A
:1006F4004C4801F07FF9BB6873B1012B04D1C8F8F1
:1007040010504FF0080909E0C8F814504FF00809D8
:1007140004E04FF0000901E04FF00409FF2C01D878
:10072400404601E008F10400FF2C01D8B30002E0C8
:10073400A6F108039B0001680F229A4021EA0202F5
:1007440009FA03F3134303607B6813F0805F00F03E
:100754008A80384B9A6942F001029A619B6903F0DE
:1007640001030193019BB1088A1C334B53F8220007
:1007740006F003039B000F229A4020EA0200284A55
:10078400904515D002F58062904513D002F5806241
:10079400904511D002F5806290450FD002F5806239
:1007A40090450DD002F5806290450BD105220AE0F8
:1007B400002208E0012206E0022204E0032202E013
:1007C400042200E0062202FA03F3034302311A4A28
:1007D40042F821307B6813F4803F05D002F5806233
:1007E40013682343136004E0144A136823EA0403E0
:1007F40013607B6813F4003F04D0104A536823430A
:10080400536004E00D4A536823EA040353607B6891
:1008140013F4801F14D0094A93682343936014E0AF
:1008240000080140E41D0008000011100000211020
:10083400000031100010024000000140000401409B
:100844000C4A936823EA040393607B6813F4001F43
:1008540004D0084AD3681C43D46004E0054AD36832
:1008640023EA0404D46001360F2E7FF6BDAE03B034
:10087400BDE8F0830004014070B5064615460C46F9
:1008840021B94FF4F271084801F0B4F8012D04D9EC
:1008940040F2E511044801F0ADF80DB1346170BDCA
:1008A4002404346170BD00BFE41D000838B504465B
:1008B4000D4621B94FF4FD71034801F09BF8E1683E
:1008C4006940E16038BD00BFE41D000830B583B065
:1008D400044620B94FF48771B94801F08BF82368B6
:1008E4003BB113F00F0F04D140F20F11B44801F0E3
:1008F40081F8236813F0010F00F0A380636853B1FB
:10090400B3F5803F07D0B3F5A02F04D040F2151102
:10091400AB4801F06FF8AB4B5B6803F00C03042B9E
:100924000AD0A84B5B6803F00C03082B1BD1A54B22
:100934005B6813F4803F16D04FF4003393FAA3F3AB
:10094400A04B1A684FF4003393FAA3F3B3FA83F37A
:1009540003F01F0322FA03F313F0010F71D063684D
:10096400002B6ED11BE36368B3F5803F05D1954A34
:10097400136843F48033136026E063B903F18043C2
:1009840003F504331A6822F480321A601A6822F4D8
:1009940080221A6018E0B3F5A02F0CD103F1804334
:1009A400A3F53C331A6842F480221A601A6842F4B0
:1009B40080321A6008E0834B1A6822F480321A608D
:1009C4001A6822F480221A606368EBB1FFF70EFD07
:1009D400054605E0FFF70AFD401B642800F2E182AA
:1009E4004FF4003393FAA3F3764B1A684FF40033B1
:1009F40093FAA3F3B3FA83F303F01F0322FA03F386
:100A040013F0010FE6D01CE0FFF7F0FC054605E00B
:100A1400FFF7ECFC401B642800F2C5824FF400335E
:100A240093FAA3F3674B1A684FF4003393FAA3F3D2
:100A3400B3FA83F303F01F0322FA03F313F0010F55
:100A4400E6D1236813F0020F00F0A0802369012B84
:100A540004D940F249115A4800F0CCFF63691F2BB6
:100A640004D94FF4A571564800F0C4FF554B5B6898
:100A740013F00C0F0AD0534B5B6803F00C03082BE4
:100A840027D1504B5B6813F4803F22D1022393FAA1
:100A9400A3F34C4B1A68022393FAA3F3B3FA83F338
:100AA40003F01F0322FA03F313F0010F03D02369A9
:100AB400012B40F07A824348036823F0F80163690C
:100AC400F82292FAA2F2B2FA82F293400B43036044
:100AD4005CE023699BB3012292FAA2F3B3FA83F395
:100AE4009B0003F1844303F584031A60FFF77EFC43
:100AF400054605E0FFF77AFC401B022800F2578206
:100B0400022393FAA3F32F4B1A68022393FAA3F355
:100B1400B3FA83F303F01F0322FA03F313F0010F74
:100B2400E8D02848036823F0F8016369F82292FAB0
:100B3400A2F2B2FA82F293400B43036026E001234F
:100B440093FAA3F3B3FA83F39B0003F1844303F50D
:100B5400840300221A60FFF749FC054605E0FFF70D
:100B640045FC401B022800F22482022393FAA3F3DB
:100B7400144B1A68022393FAA3F3B3FA83F303F032
:100B84001F0322FA03F313F0010FE8D1236813F0D3
:100B9400080F5CD0A369012B04D94FF4C571084830
:100BA40000F028FFA3696BB3012292FAA2F3B3FA0F
:100BB40083F3054941F82320FFF718FC05460BE0B1
:100BC400281E00080010024080044242FFF70EFC79
:100BD400401B022800F2EF81022393FAA3F293FA56
:100BE400A3F2A44A526A93FAA3F3B3FA83F303F089
:100BF4001F0322FA03F313F0010FE7D00120FFF7DC
:100C0400FBFB24E0012393FAA3F3B3FA83F300215B
:100C1400994A42F82310FFF7E9FB054605E0FFF780
:100C2400E5FB401B022800F2C881022393FAA3F2D9
:100C340093FAA3F28F4A526A93FAA3F3B3FA83F3B3
:100C440003F01F0322FA03F313F0010FE7D1236823
:100C540013F0040F00F0AB80E368012B06D9052BD9
:100C640004D040F2B711854800F0C4FE814BDA6924
:100C740042F08052DA61DB6903F080530193019BF7
:100C84007F4A136843F480731360FFF7AFFB054694
:100C940005E0FFF7ABFB401B642800F29081784B22
:100CA4001B6813F4807FF4D0E368012B05D1714AEB
:100CB400136A43F00103136222E063B903F1804332
:100CC40003F504331A6A22F001021A621A6A22F046
:100CD40004021A6214E0052B09D1664B1A6A42F029
:100CE40004021A621A6A42F001021A6208E0614BB5
:100CF4001A6A22F001021A621A6A22F004021A62C3
:100D0400E36853B3FFF772FB054607E0FFF76EFB9A
:100D1400401B41F28833984200F25381022393FA34
:100D2400A3F293FAA3F3B3FA83F35B0943F0020348
:100D3400DBB2022B02D14F4B1A6A01E04D4B5A6AC7
:100D4400022393FAA3F3B3FA83F303F01F0322FA03
:100D540003F313F0010FD9D029E0FFF747FB054651
:100D640007E0FFF743FB401B41F28833984200F24F
:100D74002A81022393FAA3F293FAA3F3B3FA83F337
:100D84005B0943F00203DBB2022B02D1394B1A6A2E
:100D940001E0384B5A6A022393FAA3F3B3FA83F3BC
:100DA40003F01F0322FA03F313F0010FD9D1E3690F
:100DB400022B04D940F24721304800F01BFEE369BE
:100DC400002B00F002812B4A526802F00C02082A20
:100DD40000F0FD80022B40F0B780236A3BB1B3F5ED
:100DE400803F04D04FF41471244800F003FE636A7A
:100DF40073B3B3F5802F2BD0B3F5002F28D0B3F500
:100E0400402F25D0B3F5801F22D0B3F5A01F1FD0EB
:100E1400B3F5C01F1CD0B3F5E01F19D0B3F5001F04
:100E240016D0B3F5101F13D0B3F5201F10D0B3F5AF
:100E3400301F0DD0B3F5401F0AD0B3F5501F07D0B3
:100E4400B3F5601F04D040F251210C4800F0D2FDEC
:100E54004FF0807393FAA3F3B3FA83F39B0003F187
:100E6400844303F5840300221A60FFF7BFFA0546A2
:100E74000EE000BF0010024080044242281E000819
:100E840000700040FFF7B2FA401B022800F2A18074
:100E94004FF0007393FAA3F3514B1A684FF00073A9
:100EA40093FAA3F3B3FA83F303F01F0322FA03F3D1
:100EB40013F0010FE6D1236AB3F5803F10D1A36884
:100EC4003BB1B3F5003F04D040F26721454800F040
:100ED40091FD43494B6823F40032A36813434B60EC
:100EE4003F48436823F47411236A626A13430B4333
:100EF40043604FF0807393FAA3F3B3FA83F39B0038
:100F040003F1844303F5840301221A60FFF76EFAA8
:100F1400044604E0FFF76AFA001B02285BD84FF08E
:100F2400007393FAA3F32E4B1A684FF0007393FAED
:100F3400A3F3B3FA83F303F01F0322FA03F313F0CA
:100F4400010FE7D0002049E04FF0807393FAA3F338
:100F5400B3FA83F39B0003F1844303F58403002273
:100F64001A60FFF743FA044604E0FFF73FFA001B58
:100F7400022832D84FF0007393FAA3F3184B1A687F
:100F84004FF0007393FAA3F3B3FA83F303F01F0350
:100F940022FA03F313F0010FE7D100201EE0012031
:100FA4001CE003201AE0032018E0012016E00320CF
:100FB40014E0032012E0032010E003200EE00320DD
:100FC4000CE003200AE0032008E0002006E00120F2
:100FD40004E0032002E0032000E0032003B030BD5E
:100FE40000100240281E000830B486B01F4D02AC29
:100FF40028686968AA68EB680FC42B8AADF80430C6
:101004001B4B5B6803F00C02082A2AD103F470110D
:101014004FF4701292FAA2F2B2FA82F221FA02F2B8
:1010240006A90A4412F8102C13F4803F15D0104B73
:101034005B6803F400314FF4003393FAA3F3B3FA7B
:1010440083F321FA03F306A90B4413F8140C094B98
:10105400B3FBF0F000FB02F004E0074800FB02F0F1
:1010640000E0044806B030BC704700BF141E0008FE
:101074000010024000127A0000093D0070B50D46D0
:10108400044620B94FF42F71A04800F0B3FC236844
:1010940013F00F0F04D140F2BD219C4800F0AAFCCC
:1010A400022D04D940F2BE21984800F0A3FC984BCD
:1010B4001B6803F007039D420BD9954A136823F07C
:1010C40007032B431360136803F007039D4240F0AA
:1010D4000D81236813F0020F1DD0A368A3B1802BE8
:1010E40012D0902B10D0A02B0ED0B02B0CD0C02B34
:1010F4000AD0D02B08D0E02B06D0F02B04D040F23D
:10110400D721824800F076FC82494B6823F0F00234
:10111400A36813434B60236813F0010F00F0818030
:101124006368022B04D940F2DE21784800F062FCA7
:101134006268012A13D14FF4003393FAA3F3754B79
:1011440019684FF4003393FAA3F3B3FA83F303F06B
:101154001F0321FA03F313F0010F28D1C8E0022A78
:1011640013D14FF0007393FAA3F36A4B19684FF04D
:10117400007393FAA3F3B3FA83F303F01F0321FA82
:1011840003F313F0010F12D1B4E0022393FAA3F393
:10119400604B1968022393FAA3F3B3FA83F303F0C1
:1011A4001F0321FA03F313F0010F00F0A58059493E
:1011B4004B6823F0030313434B60FFF717F906460C
:1011C4006368012B0FD107E0FFF710F9801B41F290
:1011D4008833984200F292804E4B5B6803F00C0314
:1011E400042BF1D11DE0022B16D107E0FFF7FEF826
:1011F400801B41F28833984200F28280454B5B6841
:1012040003F00C03082BF1D10BE0FFF7EFF8801B80
:1012140041F28833984275D83E4B5B6813F00C0F4B
:10122400F3D13B4B1B6803F007039D420AD2384AB3
:10123400136823F007032B431360136803F00703B9
:101244009D4261D1236813F0040F19D0E36883B180
:10125400B3F5806F0DD0B3F5A06F0AD0B3F5C06FAE
:1012640007D0B3F5E06F04D040F23231274800F0E4
:10127400C1FB28494B6823F4E062E36813434B60E5
:10128400236813F0080F1AD0236983B1B3F5806F74
:101294000DD0B3F5A06F0AD0B3F5C06F07D0B3F586
:1012A400E06F04D040F23931184800F0A3FB194A2A
:1012B400536823F46053216943EAC1035360FFF781
:1012C40093FE144B5B6803F0F002F02393FAA3F34C
:1012D400B3FA83F322FA03F30F4AD35CD8400F4BDB
:1012E40018600020FFF754F8002070BD012070BD85
:1012F400012070BD012070BD012070BD032070BDB0
:10130400032070BD032070BD012070BD281E00089D
:101314000020024000100240B01E00080C00002013
:10132400014B1868704700BF0C0000202DE9F04104
:1013340005460E4690461C46FFF758F80746B8F196
:10134400000F2AD05BE0B4F1FF3F26D024B1FFF7B1
:101354004DF8C01B844220D22A68536823F0E0036E
:1013640053602A68136823F040031360AB6AB3F533
:10137400005F09D12A68136823F4005313602A68B4
:10138400136843F400531360012385F8513000239C
:1013940085F850300320BDE8F0812B689B6836EA5D
:1013A4000303D0D10020BDE8F081B4F1FF3F26D083
:1013B40024B1FFF71BF8C01B844220D22A6853686B
:1013C40023F0E00353602A68136823F0400313609A
:1013D400AB6AB3F5005F09D12A68136823F400539C
:1013E40013602A68136843F400531360012385F8DB
:1013F4005130002385F850300320BDE8F0812B687C
:101404009B6836EA0303D0D00020BDE8F08100BF1A
:10141400F0B583B090F85150EDB2012D40F0D18079
:10142400002900F0D080002A00F0CF801F46164625
:101434000D46044683683BB1B3F5004F04D040F237
:10144400A311674800F0D6FA94F85030012B00F04D
:10145400BE80012384F85030122384F851300023D5
:1014640063652563A686E686E364A364A363A38712
:10147400E387A36AB3F5005F09D12268136823F4F4
:10148400005313602268136843F400531360A36885
:10149400B3F5004F04D12268136843F4804313600A
:1014A40023681A6812F0400F03D11A6842F0400210
:1014B4001A60E368002B2CD1636813B1E38E012B0F
:1014C4001AD12268236B591C21631B78D360E38EE5
:1014D400013BE38610E03B46002202212046FFF751
:1014E40025FF002875D12268236B591C21631B78C2
:1014F400D360E38E013BE386E38E002BEBD1A36A3A
:10150400B3F5005F33D12268136843F4805313604A
:101514002DE0636813B1E38E012B1CD12368226B89
:101524001288DA60236B02332363E38E013BE38684
:1015340011E03B46002202212046FFF7F7FE002877
:1015440049D12368226B1288DA60236B0233236348
:10155400E38E013BE386E38E002BEAD1A36AB3F565
:10156400005F04D12268136843F4805313603B4640
:10157400002202212046FFF7D9FE28B1636D43F013
:1015840010036365032327E03B46012280212046A4
:10159400FFF7CCFE034628B1636D43F01003636587
:1015A400032319E0A2682AB92268D16801919268DC
:1015B4000192019A012284F85120002284F85020DB
:1015C4000AE0022308E0012306E0012304E00223E9
:1015D40002E0032300E00323184603B0F0BD00BF7C
:1015E400541E0008002800F0BC8010B504460368AF
:1015F4005D4A93420BD0A2F57842934207D002F59C
:101604008062934203D06B21584800F0F3F9636879
:1016140033B1B3F5827F03D06C21544800F0EAF96A
:10162400A3684BB1B3F5806F06D0B3F5004F03D078
:101634006D214E4800F0DEF9E368B3F5006F04D085
:101644001BB16E21494800F0D5F923692BB1022B57
:1016540003D06F21454800F0CDF96369012B03D90C
:101664007021424800F0C6F9A369B3F5007F07D0A2
:1016740033B1B3F5802F03D071213C4800F0BAF99F
:10168400E3698BB1082B0FD0102B0DD0182B0BD086
:10169400202B09D0282B07D0302B05D0382B03D092
:1016A4007221324800F0A6F9236A2BB1802B03D0B3
:1016B40073212E4800F09EF9636A1BB174212B48F4
:1016C40000F098F9A36A33B1B3F5005F03D0752134
:1016D400264800F08FF9E36A013B4FF6FE7293420D
:1016E40003D97621214800F085F994F8513013F09C
:1016F400FF0F02D1204600F0C7F9022384F85130CD
:101704002268136823F04003136021686268A368A9
:101714001A43E3681A4323691A4363691A43A369A2
:1017240003F400731343E2691343226A1343A26A66
:101734001A430A602168638B03F00402636A13434B
:101744004B602368E26A1A612268D36923F4006358
:10175400D3610020064B18706065012384F8513072
:1017640010BD0120704700BF00300140801E0008FA
:101774001C000020FEE700BF01230360014B0B6047
:10178400704700BF0400002008B500F00FF8024BBA
:10179400024A9A6008BD00BF00ED00E000000008A6
:1017A40008B500F029F808BDFEE700000F4B1A68E1
:1017B40042F001021A6059680D4A0A405A601A68D8
:1017C40022F0847222F480321A601A6822F4802291
:1017D4001A605A6822F4FE025A604FF41F029A609B
:1017E4004FF00062034B9A60704700BF0010024044
:1017F4000000FFF800ED00E01F4B5B6803F00C03F2
:10180400042B06D0082B08D03BBB1C4A1C4B1A6087
:1018140026E01A4A1A4B1A6022E0174A53685268A3
:10182400C3F38343023312F4803F05D1154A02FB0C
:1018340003F3134A136013E00F4A526812F4003F93
:1018440005D0104A02FB03F30D4A136008E00B4A6B
:1018540002FB03F30A4A136002E0084A084B1A60C9
:10186400054B5B68C3F30313074AD15C044A13684E
:10187400CB401360704700BF0010024000127A0092
:101884000C00002000093D00B01E0008F0B587B030
:101894001C4B9A6942F010029A619A6902F0100294
:1018A4000092009A9A6942F004029A619B6903F0DB
:1018B40004030193019B144F00224FF40051384656
:1018C400FEF7DAFF114C002206212046FEF7D4FF72
:1018D400012208212046FEF7CFFF4FF40053029364
:1018E400012603960225059502A93846FEF728FE2F
:1018F4000E2302930396059502A92046FEF720FEC7
:1019040007B0F0BD00100240001001400008014083
:1019140008B500F01DF9FEE708B50E480E4B03604C
:101924004FF48273436000238360C3600222026128
:10193400012242614FF4007282611822C261036283
:10194400436283620A23C362FFF74CFE08B1FFF7C8
:10195400DFFF08BD240000200030014000B591B035
:10196400012306934FF48033079300220892022246
:101974000D920E934FF4E0130F9306A8FEF7A6FF03
:1019840008B1FFF7C5FF0F23019302210291002341
:1019940003934FF480620492059301A8FFF76EFB52
:1019A40008B1FFF7B5FFFFF7BBFC094BA3FB003001
:1019B4008009FEF78FFD0420FEF7A2FD00221146E8
:1019C4004FF0FF30FEF744FD11B05DF804FB00BF9B
:1019D400D34D621008B500F0AFF8FEF7EDFCFFF749
:1019E400BDFFFFF753FFFFF797FF00F0B3F800F0D8
:1019F400A7F8FCE7704700BF00B583B0204B9A6995
:101A040042F001029A619B6903F001030193019B77
:101A14000320FEF7FFFC002211466FF00B00FEF7D7
:101A240017FD002211466FF00A00FEF711FD002297
:101A340011466FF00900FEF70BFD002211466FF00E
:101A44000400FEF705FD002211466FF00300FEF7C7
:101A5400FFFC002211466FF00100FEF7F9FC0022A2
:101A640011464FF0FF30FEF7F3FC064A536823F0AB
:101A7400E06343F00073536003B05DF804FB00BF00
:101A840000100240000001400268134B9A4222D128
:101A940010B586B003F560439A6942F480529A61A6
:101AA4009B6903F480530193019BA02302930223B7
:101AB400039303230593094C02A92046FEF740FD36
:101AC4004023029300230393049302A92046FEF7C4
:101AD40037FD06B010BD70470030014000080140DA
:101AE400704700BFFEE700BFFEE700BFFEE700BF90
:101AF400FEE700BF704700BF704700BF704700BFDC
:101B040008B5FEF76BFCFEF717FD08BD08B54FF4EA
:101B140000510248FEF7CAFE08BD00BF0010014094
:101B240008B54FF47A7300221146024800F0CAF84F
:101B340008BD00BF111B000808B500F0ABF808BDD4
:101B440008B500F0DFF808BD08B500F007F908BDD6
:101B5400704700BF08B5FFF7E3FF034A00210846BA
:101B640000F058F808BD00BFC01E000808B50246C2
:101B740002210248FEF780FE08BD00BF00080140B4
:101B840008B5024608210248FEF776FE08BD00BFEC
:101B94000008014010B582B002AC04F8010D002029
:101BA400FFF7EEFF0120FFF7E1FF002301222146AA
:101BB4000348FFF72DFC0120FFF7E2FF02B010BD40
:101BC4002400002010B582B002AC04F8010D0020FE
:101BD400FFF7D6FF0020FFF7C9FF002301222146AB
:101BE4000348FFF715FC0120FFF7CAFF02B010BD40
:101BF4002400002010B504465039C8B2FFF7E2FFB4
:101C0400200940F01000FFF7DDFF04F00F00FFF79C
:101C1400D9FF10BD2DE9F8430646884691460027B2
:101C24002FE0203DEDB2782E04D908F101085FFAC7
:101C340088F8002641463046FFF7DCFF002407E021
:101C440004EB0513124AD05CFFF7A4FF0134E4B29D
:101C5400072CF5D908F10101C9B23046FFF7CAFFD4
:101C6400002408E004EB05130833094AD05CFFF7AD
:101C740091FF0134E4B2072CF4D90836F6B20137E7
:101C8400FFB219F90750002DCBD1BDE8F88300BF8E
:101C9400C81E000830B400230EE0094C9900CA188D
:101CA400950060190022625142600272C2602846A7
:101CB400204402610133DBB20F2BEED930BC7047F4
:101CC4007C000020F0B5002417E0274604EB8406CE
:101CD400B5000B4E3544ED686DB934464FEA870EB6
:101CE4000EEB0705AE00A519A2516B6000232B7201
:101CF400E8602961F0BD0134E4B20F2CE5D9F0BDF0
:101D04007C00002070B5002422E004EB84029300E0
:101D1400114A1344DB68CBB104EB840293000E4AEE
:101D240013441B7A93B1A10021448A000A4E16443D
:101D3400013B3372F36830699847736833B904EB35
:101D44008405AB00044A13440022DA600134E4B28F
:101D54000F2CDAD970BD00BF7C00002070B40023C2
:101D64001FE003EB8300820010480244D268B2B142
:101D740003EB830082000D48825852B904469A004E
:101D8400D518A80025186E682650287A411C297297
:101D940005E003EB83018800013A04490A5001334A
:101DA400DBB20F2BDDD970BC704700BF7C00002074
:101DB4002E2E2F73797374656D2F7372632F737462
:101DC4006D3332663178782F73746D3332663178BF
:101DD400785F68616C5F636F727465782E6300006E
:101DE4002E2E2F73797374656D2F7372632F737432
:101DF4006D3332663178782F73746D33326631788F
:101E0400785F68616C5F6770696F2E630000000023
:101E140002030405060708090A0B0C0D0E0F101027
:101E2400010200002E2E2F73797374656D2F737267
:101E3400632F73746D3332663178782F73746D3316
:101E440032663178785F68616C5F7263632E630019
:101E54002E2E2F73797374656D2F7372632F7374C1
:101E64006D3332663178782F73746D33326631781E
:101E7400785F68616C5F7370692E63002E2E2F7318
:101E8400797374656D2F7372632F73746D33326657
:101E94003178782F73746D3332663178785F686186
:101EA4006C5F7370695F65782E630000000000004A
:101EB40000000000010203040607080948616C6C75
:101EC4006F0000000000000000000000000000009F
:101ED40000000000000000F80000000000000033D3
:101EE4003000000000100C06100C0600000000007A
:101EF4000000000040C07840C0784000043F040463
:101F04003F040400007088FC08300000001820FF23
:101F1400211E0000F008F000E018000000211C035E
:101F24001E211E0000F00888700000001E212324DA
:101F34001927211010160E000000000000000000F8
:101F440000000000000000E0180402000000000788
:101F54001820400000020418E0000000004020188F
:101F640007000000404080F0804040000202010F62
:101F740001020200000000F0000000000101011F46
:101F840001010100000000000000000080B07000AA
:101F9400000000000000000000000000000101013A
:101FA40001010101000000000000000000303000C9
:101FB40000000000000000008060180400601806A3
:101FC4000100000000E010080810E000000F1020DD
:101FD40020100F00001010F8000000000020203F27
:101FE40020200000007008080888700000302824B1
:101FF4002221300000300888884830000018202052
:1020040020110E000000C02010F800000007042476
:10201400243F240000F808888808080000192120BB
:1020240020110E0000E0108888180000000F112015
:1020340020110E0000380808C83808000000003FCE
:10204400000000000070880808887000001C22212D
:1020540021221C0000E010080810E00000003122DA
:1020640022110F00000000C0C0000000000000307A
:1020740030000000000000800000000000008060CC
:10208400000000000000804020100800000102044D
:102094000810200040404040404040000404040434
:1020A40004040400000810204080000000201008F0
:1020B40004020100007048080808F0000000003025
:1020C40036010000C030C828E810E00007182724B3
:1020D40023140B000000C038E0000000203C230261
:1020E4000227382008F8888888700000203F2020C4
:1020F40020110E00C03008080808380007182020F6
:102104002010080008F808080810E000203F2020EC
:1021140020100F0008F88888E8081000203F2020CD
:102124002320180008F88888E8081000203F2000C1
:1021340003000000C03008080838000007182020F9
:10214400221E020008F808000008F808203F2101B8
:1021540001213F20000808F8080800000020203F63
:102164002020000000000808F8080800C0808080D3
:102174007F00000008F888C028180800203F2001CC
:102184002638200008F8080000000000203F202026
:102194002020300008F8F800F8F80800203F003F3D
:1021A400003F200008F830C00008F808203F200055
:1021B40007183F00E01008080810E0000F10202066
:1021C40020100F0008F808080808F000203F21013B
:1021D40001010000E01008080810E0000F18242492
:1021E40038504F0008F8888888887000203F200005
:1021F400030C3020007088080808380000382021BB
:1022040021221C00180808F8080818000000203FC4
:102214002000000008F808000008F808001F20202B
:1022240020201F000878880000C8380800000738FC
:102234000E010000F80800F80008F800033C07004D
:10224400073C0300081868808068180820302C03B5
:10225400032C30200838C800C83808000000203F8C
:102264002000000010080808C8380800203826217B
:1022740020201800000000FE020202000000007F7F
:1022840040404000000C30C000000000000000018D
:102294000638C00000020202FE0000000040404078
:1022A4007F0000000000040202020400000000009D
:1022B400000000000000000000000000808080801A
:1022C4008080808000020204000000000000000002
:1022D400000000000000808080800000001924229B
:1022E40022223F2008F8008080000000003F1120D7
:1022F40020110E000000008080800000000E1120DC
:1023040020201100000000808088F800000E1120B9
:1023140020103F200000808080800000001F2222C7
:1023240022221300008080F0888888180020203F33
:10233400202000000000808080808000006B949446
:102344009493600008F8008080800000203F210002
:1023540000203F2000809898000000000020203FCB
:1023640020200000000000809898000000C08080B9
:10237400807F000008F8000080808000203F240255
:102384002D302000000808F8000000000020203F45
:10239400202000008080808080808000203F2000FA
:1023A4003F20003F8080008080800000203F21008B
:1023B40000203F200000808080800000001F20203B
:1023C40020201F00808000808000000080FFA1206A
:1023D40020110E000000008080808000000E11207B
:1023E40020A0FF80808080008080800020203F210A
:1023F40020000100000080808080800000332424BD
:1024040024241900008080E0808000000000001F68
:10241400202000008080000000808000001F202019
:1024240020103F20808080000080808000010E30DA
:102434000806010080800080008080800F300C033B
:102444000C300F0000808000808080000020312E3E
:102454000E312000808080000080808080818E701A
:102464001806010000808080808080000021302CCC
:102474002221300000000000807C020200000000E5
:10248400003F404000000000FF000000000000008A
:10249400FF0000000002027C800000000040403F7A
:1024A4000000000000060101020204040000000014
:0424B4000000000024
:1024B80078563412200000200000000000A24A04D0
:0424C800325476987C
:04000005080001E509
:00000001FF
